:100000000C94B8030C94F0030C94F0030C94F003DC
:100010000C94F0030C94F0030C94F0030C94F00394
:100020000C94F0030C94F0030C94691D0C94A51C23
:100030000C94A8170C94F0030C94F0030C94F003A8
:100040000C94F0030C94F0030C94F0030C94F00364
:100050000C94F0030C9467170C94F0030C94F003C9
:100060000C94F0030C94F0030C94F0030C94F00344
:100070000C94F0030C94F0030C94F0030C94F00334
:100080000C94F0030C94F0030C94F0030C94F00324
:100090000C94F0030C94F0030C94F0030C94F00314
:1000A0000C94F0030C94F0030C94F0033C083C080F
:1000B0006E086E08E008FC08930A930A0709E50930
:1000C000F609F609BE1AE51A7D1CE51A7D1C2D1BE2
:1000D000501B7D1C3F1C521C29003A003C003E0076
:1000E0004000420044004600480000003B003D0044
:1000F0003F004100430045004700000035001F005D
:1001000021002300250027002E0049004B001E007F
:1001100020002200240026002D002A004A000000B2
:100120002B001A0015001C000C00130030004C00BE
:100130004E00140008001700180012002F003100B4
:100140004D0000003900160009000B000E003300BE
:100150002A0000000000040007000A000D000F0044
:100160003400280000000000E1001D00060005002A
:1001700010003700E5000000000031001B001900EE
:10018000110036003800015152000000E000E2008A
:100190000000050000000000E70050004F00E300F1
:1001A00000002C0000002C00E600E40051000000DC
:1001B000010001000100C35CC75CC95CCB5CC05C92
:1001C000BF5C000001000100C45CC65CC85CCA5C86
:1001D000BE5C0000010001000100010001000100FF
:1001E0000100010001000100010001000100010007
:1001F00001000100010000000100010001000100F8
:1002000001000100010001000100010001000100E6
:1002100001000100010001000100000001000100D7
:1002200001000100010001000100000000000100C8
:1002300001000100010001000100010000000000B8
:1002400001000100010001000100010001000000A7
:100250000000010001000100010001000100010097
:10026000010000000100010000000100000000008A
:100270000100010001000100000001000000025126
:100280000100010001000000010001000100010067
:100290000100010001000100010000000100010057
:1002A0000100010001000100010000000100010047
:1002B0000100010001000100010001000100010036
:1002C0000100010001000100010001000100000027
:1002D00001000100005C01000100010001000100BB
:1002E0000100010001000100010001000100010006
:1002F00001000000010001000100010001000100F7
:1003000001000000000001000100010001000100E7
:1003100001000100000000000100010001000100D7
:1003200001000100010000000000010001000100C7
:1003300001000100010001000100000001000100B6
:1003400000000100000000000100010001000100A8
:100350000000010000000100010001000100000098
:100360000100010001000100010001000100010085
:100370000100000001000100010001000100010076
:100380000100000001000100010001000100010066
:100390000100010001000100010001000100010055
:1003A0000100010001000000010001000100010046
:1003B0000100010001000100010001000100010035
:1003C0000100010001000100010000000100010026
:1003D0000100010001000100010000000000010017
:1003E0000100010001000100010001000000000007
:1003F00001000100010001000100010001000000F6
:1004000000000100010001000100010001000100E5
:1004100001000000010001000000010000000000D8
:1004200001000100010001000000010000000100C6
:10043000010001000100000000047F3F1F6432142E
:10044000783C1E1E140A052223252628292A2C2D35
:100450002F3032333536383A3B3D3E4042434547F4
:10046000494A4C4E5051535557595A5C5E6062642C
:100470006668696B6D6F71737577797B7D7F81833A
:100480008587898A8C8E90929496989A9C9E9FA13B
:10049000A3A5A7A8AAACAEAFB1B3B4B6B8B9BBBC5C
:1004A000BEBFC1C2C3C5C6C7C9CACBCCCDCED0D1D1
:1004B000D2D2D3D4D5D6D7D7D8D9D9DADADBDBDBC9
:1004C000DCDCDCDCDCDDDDDDDDDCDCDCDCDCDBDB6A
:1004D000DBDADAD9D9D8D7D7D6D5D4D3D2D2D1D0BE
:1004E000CECDCCCBCAC9C7C6C5C3C2C1BFBEBCBBBB
:1004F000B9B8B6B4B3B1AFAEACAAA8A7A5A3A19F33
:100500009E9C9A98969492908E8C8A8987858381F6
:100510007F7D7B79777573716F6D6B6968666462D7
:10052000605E5C5A5957555351504E4C4A494745A5
:100530004342403E3D3B3A3836353332302F2D2C46
:100540002A29282625232205010902A1018502095D
:1005500001A1000509190129081500250195087553
:100560000181020501093009311581257F95027548
:1005700008810609381581257F95017508810605D2
:100580000C0A38021581257F950175088106C0C0C7
:1005900005010980A101850319012AB7001501266B
:1005A000B700950175108100C0050C0901A10185F6
:1005B0000419012AA002150126A0029501751081D7
:1005C00000C005010906A101050719E029E715008A
:1005D00025019508750181029501750881010507BE
:1005E000190029FF150026FF0095067508810005F2
:1005F0000819012905950575019102950175039169
:1006000001C009023B00020100A0FA090400000138
:1006100003010100092111010001224000070581A9
:100620000308000109040100010300000009211171
:10063000010001227B000705820320000112010056
:100640000200000008584647560100010200010C54
:100650000356006900720067006F0000000803463F
:10066000004C0058000000040309040001010101CE
:10067000010101010102020202020202020203035D
:10068000030303030303040404040404040505052D
:1006900005050606060606070707070708080808EF
:1006A000090909090A0A0A0B0B0B0C0C0C0D0D0D9C
:1006B0000E0E0E0F0F0F1010111111121213131432
:1006C00014151516161717181819191A1A1B1B1CAA
:1006D0001D1D1E1E1F202021222223242425262604
:1006E000272829292A2B2C2D2D2E2F303132323339
:1006F0003435363738393A3B3C3D3E3F4041424342
:100700004445464748494A4C4D4E4F505153545525
:100710005658595A5B5D5E5F616264656668696BD5
:100720006C6D6F7072737577787A7B7D7E80828353
:100730008587888A8C8E8F91939596989A9C9EA097
:10074000A2A3A5A7A9ABADAFB1B3B5B7BABCBEC0A4
:10075000C2C4C6C9CBCDCFD1D4D6D8DBDDDFE2E46D
:10076000E7E9EBEEF0F3F5F8FAFDFFFFAA7F55405D
:1007700011241FBECFEFDAE0DEBFCDBF04B603FE0B
:1007800018C08091B4029091B502A091B602B091C8
:10079000B7028730904BA740B04B59F41092B40287
:1007A0001092B5021092B6021092B702E0E0F8E3A0
:1007B000099511E0A0E0B1E0E0EEF8E402C0059098
:1007C0000D92A038B107D9F722E0A0E8B1E001C04E
:1007D0001D92A43BB207E1F70E9497110C946E247E
:1007E0000C9400001F93CF93DF93CDB7DEB76797CC
:1007F0000FB6F894DEBF0FBECDBF4B8B5C8B6D8BFD
:100800007E8B8F8B61111092CC0186E09E01235F5D
:100810003F4FD901E82F1D92EA95E9F795E0FE01D7
:100820007396D90101900D929A95E1F79C894E89B2
:100830005F897B897D879E876F87598B488BF901FC
:10084000DE01179601900D928A95E1F7CE01079689
:100850000E94F60F81113EC086E0FE013796DE0150
:10086000119601900D928A95E1F7FF81E8856A85DE
:100870007B856115710531F0EF3F31F481E0FF3F79
:1008800019F403C081E001C080E080FD23C0209105
:10089000910130E0C9010196877099274091C2010A
:1008A00050E08417950779F1F983EA837D836C839F
:1008B00096E0929FD001939FB00D1124AE56BE4F8B
:1008C000FE01319601900D929A95E1F78093910186
:1008D0000E94640F16E08091C201909191018917E6
:1008E000F9F0189FC00111248E569E4F0E94F60FFA
:1008F0008823B1F08091C20190E00196877099271A
:100900008093C201E8CF0E94DF22109291011092E1
:10091000C201EBE8F1E086E0DF011D928A95E9F77C
:1009200067960FB6F894DEBF0FBECDBFDF91CF91B3
:100930001F91089582FB992790F981FD02C0769A54
:1009400001C07698911102C02A9A08952A980895B4
:100950008F929F92AF92BF92CF92DF92EF92FF92CF
:100960000F931F93CF93DF93CDB7DEB72A970FB6C0
:10097000F894DEBF0FBECDBFFC010081D180838122
:100980009481892B39F01FEFD11206C091E00F3FFF
:1009900019F403C091E001C090E090FDC8C67F014A
:1009A00085E0DE01169601900D928A95E1F7F70138
:1009B00022818E819F81222349F00E94B521182F28
:1009C000682F8E819F810E943A2203C00E940E22CE
:1009D000182F99E02CE6129FF00111249D9DE00D47
:1009E000F11D1124E00FF11DEE0FFF1FE852FF4F24
:1009F00005911491F7018281882309F4A3C00E3B6D
:100A0000FCE51F07B1F188F40C3B3CE51307C9F086
:100A10000D3B9CE5190709F095C080913002877065
:100A20008E7F8093300280E01DC0003CECE51E0705
:100A300009F46EC008F453C0013C2CE5120749F1DB
:100A400081C0809130028770886280933002887FF5
:100A500091E009F490E08091300290FB80F980935E
:100A6000300285E00E94AE18809130020E94611928
:100A700072C280913002982F96959695969549F17D
:100A8000915E990F990F990F8770892B809330028F
:100A900014C090913002892F8695869586958F5F38
:100AA0008F719770863008F04AC0880F880F880FC2
:100AB000892B8093300280913002887F91E009F485
:100AC00090E08091300290FB80F9809330020E9488
:100AD00061198091300286958695869523C0209174
:100AE0003002822F869586958695482F50E04530B6
:100AF000510554F48F5F982F990F990F990F822FFA
:100B00008770892B80933002809130028160DDCF25
:100B10008091300280FF09C08E7F809330020E9456
:100B2000611980E00E94AE1816C281608093300285
:100B3000813011F49093300280913002C8CF9093AD
:100B40003002B9CF043F2CE5120749F406E221EE4A
:100B500040EE64EF7CE5C7010E942318FCC1053F0D
:100B60003CE5130708F066C1093D9CE5190731F41F
:100B700007E225EE45EE69ED7CE5EDCF0A3DECE5BB
:100B80001E0731F408E221E045EE6AED7CE5E3CF93
:100B9000083DFCE51F0731F406E221EE41EE68ED69
:100BA0007CE5D9CF882309F47AC11092330204304E
:100BB0003DE5130758F40B3F8CE5180780F4C80196
:100BC00082509C45449708F054C109C002369DE507
:100BD000190729F0063AEDE51E0709F04AC10E94FF
:100BE000650E9093F3018093F2010131FCE51F073C
:100BF00009F4C6C008F042C009303CE5130709F407
:100C00009BC000F505309CE5190709F485C078F410
:100C10000330FCE51F0709F478C008F07AC0023001
:100C20001C4509F0F7C08091F2018160F1C00730E6
:100C30008CE5180709F478C008F07AC08091F201B9
:100C40008061E6C00D30ECE51E0709F487C058F45A
:100C50000B302CE5120709F479C008F07BC08091B5
:100C6000F20188606FC00F308CE5180709F480C06E
:100C700008F082C08091F201877FCAC00E3FECE588
:100C80001E0709F471C000F505312CE5120709F4BF
:100C900085C068F403318CE5180709F475C008F0C5
:100CA00095C00E94DF228091F2018F77B1C00C3F86
:100CB000ECE51E07A9F108F054C00B3F1C4509F0F4
:100CC000A9C08091F30140C002303DE5130709F44B
:100CD00089C058F401159DE5190709F45AC008F0B8
:100CE00069C08091F30182602FC00236FDE51F07C5
:100CF00009F47EC0063A2DE5120709F483C00330DB
:100D00001D4509F087C060E06EC08091F2018260ED
:100D10007FC08091F20116C08091F201886078C096
:100D20008091F30182604FC08091F201806270C0B7
:100D30008091F20180646CC00E94DF228091F201F8
:100D4000806866C0846064C081603DC08091F201AB
:100D50008E7F5EC08091F2018D7F5AC08091F2013A
:100D600016C08091F30118C08091F3018D7F2BC0D4
:100D70008091F2018F7E4CC08091F2018F7D48C03E
:100D80008091F2018F7B44C08091F201877F8B7F3D
:100D90003FC08091F3018D7F8E7F15C08091F2015D
:100DA00082FB222720F991E0922790FB82F990FBA9
:100DB00083F92EC08091F301982F909591708E7FCA
:100DC000892B90FB81F98093F30124C00E94DF22DC
:100DD0008091F20187FB222720F991E0922790FB76
:100DE00087F916C061E08EE090E00E94A62312C051
:100DF0008091F20184FB222720F991E0922790FB59
:100E000084F906C08091F201982F909590FB80F9AB
:100E10008093F2016091F2011091F30184E090E07F
:100E20000E94A623612F82E290E00E94A6230E94E6
:100E3000DF2291C0063F2CE5120731F406E221EED5
:100E400042EE66EF7CE587CE063F3CE5130730F4C3
:100E500007E225EE44EE65EF7CE57DCE073F9CE59D
:100E6000190709F09FCE07E225EE46EE67EF7CE515
:100E700072CE0631ECE51E0761F58091CD018A7ACC
:100E800091E009F490E090938201882311F065E3EA
:100E900001C069E283E891E00E94D11717C00631D2
:100EA000FCE51F0709F049C080918201882309F4FD
:100EB00079C385E3E3E8F1E029E831E09281891321
:100EC00001C0128231962E173F07C1F70E94EE0E25
:100ED00042C00B35FDE51F0751F158F401153CE503
:100EE0001307B9F00F3D1C4509F06AC00E94760E49
:100EF00032C00C359DE51907E1F00D351D4509F0AF
:100F00005FC08091F30182FB882780F991E08927F7
:100F100011C00E94DF22FFEF04E31CE0F15000400B
:100F20001040E1F700C000000E94431714C081E0A8
:100F300001C080E00E94470F43C08091CD018272C2
:100F40000D3C9CE5190709F4D5C340F1023D8CE541
:100F5000180709F059C38091C301877009F4E7C3EA
:100F6000F7018281882309F4E2C38091F30182FDB5
:100F7000DEC382E02A960FB6F894DEBF0FBECDBF67
:100F8000DF91CF911F910F91FF90EF90DF90CF9065
:100F9000BF90AF909F908F900C942A0F073CFCE578
:100FA0001F0709F493C308F00DC3043C3CE5130785
:100FB00009F482C308F0F8C2033C1C4509F457C386
:100FC000F70182810081D180882359F0802F9D2DE7
:100FD0000E94B521182F682F802F9D2D0E943A2244
:100FE00005C0802F9D2D0E940E22182F2CE6129FE7
:100FF000F001112439E0D39EE00DF11D1124E00F22
:10100000F11DEE0FFF1FE852FF4F859194910E9452
:10101000CB0C8C01982EF701D280A580A2943FE0E2
:10102000A3228091C3018770B9F0DD20A9F0812F40
:10103000807F803421F080E2800F883068F08091DA
:10104000F30182FD09C082E00E942A0F8091C30152
:101050008770CC24C3948111C12CB12EB2949FE02F
:10106000B9228B2D90E08C30910508F05CC2FC0118
:10107000EA5AFF4F0C943424812F807F1F708823FD
:1010800011F01295107FDD20B9F0112309F438C258
:1010900080E2800F883010F0911006C08091CD0161
:1010A000182B1093CD0105C08091CC01182B109303
:1010B000CC010E94EE0E24C2802F0E94FB2211233D
:1010C00009F431C2005E083078F1992069F1109579
:1010D0008091CC0118231093CC0129C0812F807FEF
:1010E0001F70803211F01295107F992021F0F1E0ED
:1010F0009F16D9F149C08091F30182FF1BC0DD200A
:1011000069F0112339F08091CD01182B1093CD0196
:101110000E94EE0E80E00E94332305C280E00E9410
:10112000FB22112309F4FFC1812F0E94E70E0E94C8
:10113000EE0EF9C1DD2081F08091CE01AA2051F0A0
:1011400001E0A01207C0182B181709F4ECC1109386
:10115000CE01E9C1812B10C0AA2021F021E0A21606
:1011600009F4E1C10E94E10E27C0DD2041F035E025
:101170003A1508F4D8C1812F0E94F122D4C184E02D
:101180008A1508F4D0C118C0DD2049F0AA2099F3CF
:10119000F701858180FFB4C18F708583ECCFAA20D1
:1011A00059F0093309F0BCC1FFEF17EE23E0F1500D
:1011B00010402040E1F7B2C1812F0E94EA22B3C162
:1011C000812F86958695837019F0813059F0ABC1D7
:1011D000DD2019F0C801937002C080E090E00E9409
:1011E0000118A9C1DD2019F0C801937002C080E088
:1011F00090E00E94EB179FC1802FDD2019F00E9424
:101200003F2102C00E9486200E945C2094C1812F51
:10121000837009F069C0D1108AC1902F929596957C
:101220009770990F990F802F8F70882E912CA12C79
:10123000B12C092E04C0880C991CAA1CBB1C0A9452
:10124000D2F704FF12C04FE050E060E070E004C04D
:10125000440F551F661F771F9A95D2F7DB01CA010D
:1012600080959095A095B09503C080E090E0DC015A
:1012700016951695412F4370423019F1C8F400912C
:10128000CF011091D0012091D1013091D201413094
:1012900059F088299929AA29BB29BC01CD016023CD
:1012A0007123822393230AC0802A912AA22AB32A77
:1012B000BC01CD01682979298A299B290E94B52280
:1012C00036C188299929AA29BB290091CF011091FB
:1012D000D0012091D1013091D201BC01CD01602714
:1012E000712782279327EACFDD2019F0812F8170A3
:1012F00001C08695882309F41AC1902F929596957E
:101300009770990F990F802F8F70882E912CA12C98
:10131000B12C092E04C0880C991CAA1CBB1C0A9471
:10132000D2F704FF12C04FE050E060E070E004C06C
:10133000440F551F661F771F9A95D2F7DB01CA012C
:1013400080959095A095B09503C080E090E0DC0179
:1013500016951695412F43704230D9F068F50091EB
:10136000EE011091EF012091F0013091F101413037
:1013700059F088299929AA29BB29BC01CD016023EC
:101380007123822393231EC0802A912AA22AB32A82
:1013900013C088299929AA29BB290091EE0110912F
:1013A000EF012091F0013091F101BC01CD016027E6
:1013B00071278227932706C0BC01CD0168297929AE
:1013C0008A299B290E946522B2C01F70DD2039F056
:1013D000812F0E949422802F0E94F122A8C0802F8A
:1013E0000E94EA22812F0E946F22A1C0802F32EF3B
:1013F000931609F443C0391538F090EF991659F057
:10140000E1EF9E16B1F177C0F3EF9F16F1F124EFF3
:10141000921659F170C0DD2019F134E03A1508F444
:1014200082C01F7181E090E0A0E0B0E0AC01BD019E
:1014300004C0440F551F661F771F1A95D2F780917D
:10144000EE019091EF01A091F001B091F1018A01BC
:101450009B01082719272A273B27C901B80129C062
:1014600025E02A1508F45FC0DCCF8091F30182FFEC
:1014700023C0DD2029F0812F8F7130C0DD20D9F30A
:10148000812F8F710E946F224EC0DD2079F01F7175
:1014900081E090E0A0E0B0E0BC01CD0104C0660FA7
:1014A000771F881F991F1A95D2F703C060E070E07C
:1014B000CB010E94652237C0DD2099F01F71812F7A
:1014C0000E9494228091F30182FD07C038E0139FAF
:1014D000C001112483608093C301812F0E94942254
:1014E00022C081E00E942A0F81E08A15E0F482E0A8
:1014F0000E942A0F18C0DD2029F0AA2009F4BBCFD2
:10150000802F09CEAA2009F4BBCF893349F49FEF7D
:10151000E7EEF3E09150E040F040E1F700C000005A
:10152000802F0E94FB2288EF8B0D843020F40E94D4
:1015300017180E949A04CC20A9F08091C30180FD65
:1015400011C0F70112828595859585950E94942298
:10155000C7010E94A8048091C30185958595859552
:101560000E946F2285E0F701DE01119601900D9235
:101570008A95E1F789819A810E940E229A810CE670
:10158000809FF001112419E0919FE00DF11D1124BD
:101590008981E80FF11DEE0FFF1FE852FF4F859183
:1015A0009491C5C089E286CC053CFCE51F0709F48F
:1015B00088C0063C1C4509F003CD4CEF5FE165E0B7
:1015C00070E29CC00A3C3CE5130709F489C070F442
:1015D000083CECE51E0709F47EC0093C1C4509F0F7
:1015E000EFCC40EF5FE164EE7FE188C00B3C2CE57F
:1015F000120709F47AC00C3C1C4509F0E1CC4EE816
:101600005EE16FE97EE17AC0033D9CE5190798F43D
:101610000F3CECE51E0709F477C008F472C0003DEA
:101620002CE5120709F473C0013D1C4509F0C8CC34
:101630006EE089E074C0053D8CE5180709F46DC0C3
:1016400060F4033DECE51E0709F464C0043D1C454D
:1016500009F0B6CC61E082E167C0063D2CE51207D7
:1016600009F460C00E351D4509F475CCA9CC8091F4
:101670002B0280FF1BC08E7F80932B0260912B0278
:1016800070912C0280912D0290912E020E947C1E5E
:1016900010926D028FEF90E7E2E081509040E040C1
:1016A000E1F700C000000E94561E55CC8160809377
:1016B0002B0261E0869538C049E450E262E570E2B1
:1016C0001DC042E550E269E470E218C045E050E216
:1016D0006CEF7FE113C044EE5FE160EF7FE10EC08D
:1016E0004CEC5FE168ED7FE109C048ED5FE16CEC37
:1016F0007FE104C04FE95EE16EE87EE10E94A61939
:101700002ACC61E081E010C065E082E008C068E0BA
:1017100086E005C061E18FE002C06CE183E10E94D8
:10172000941919CC61E08DE10E940E2014CC2A9608
:101730000FB6F894DEBF0FBECDBFDF91CF911F91E2
:101740000F91FF90EF90DF90CF90BF90AF909F9060
:101750008F90089580E008959091F20192FF0DC05E
:10176000282F2871283019F4877F846006C0282F1D
:101770002471243011F48B7F886093FF0DC0282FD3
:101780002871283119F4877E846106C0282F2471BE
:10179000243111F48B7E88612091F30120FF0DC06C
:1017A000382F3871383019F4877F816006C0382FA0
:1017B0003171313011F48E7F886021FF0DC0282FE8
:1017C0002871283119F4877E816106C0282F217184
:1017D000213111F48E7E886194FD877E0895F894FE
:1017E000E82FE295EF70F0E031A1282F2F7081E013
:1017F00090E001C0880F2A95EAF7982F90959323DF
:1018000091A392A1892B82A3789408958F929F929D
:10181000AF92BF92CF92DF92EF92FF920F931F93FE
:10182000CF93DF93CDB7DEB768970FB6F894DEBFDE
:101830000FBECDBFAE014F5F5F4F7A0188E1FA0165
:1018400011928A95E9F70CE411E06A01AA24A394A5
:10185000B12CF80180818F3F09F447C0F894E82F3C
:10186000E295EF70F0E021A18F70A50102C0440F56
:10187000551F8A95E2F7CA01922F982B91A392A146
:101880008095892382A3789400C0E8E5F1E021E007
:1018900030E0812C912C41914F3F89F0A42FA295EB
:1018A000AF70B0E090968C9190E04F7002C095952B
:1018B00087954A95E2F780FD02C0C90102C080E029
:1018C00090E0882A992A220F331F51E0E136F5076C
:1018D00011F7F80180818F3F11F00E94EF0BF0EAC1
:1018E000FA95F1F7F601918280820F5F1F4FF2E0C7
:1018F000CF0ED11C41E00835140709F0AACF48E10A
:1019000050E0B70186ED91E00E94612411E000975C
:1019100009F410E0892B89F088E1F701A6EDB1E028
:1019200001900D928A95E1F781E08093D5010E94A4
:101930009C179093D4018093D3018091D501882383
:10194000B1F08091D3019091D4010E948D17059739
:1019500070F0E6EDF1E0A7EFB1E0819191918D9308
:101960009D9351E0EE3EF507C1F71092D501812F0E
:1019700068960FB6F894DEBF0FBECDBFDF91CF9152
:101980001F910F91FF90EF90DF90CF90BF90AF909D
:101990009F908F900895CF93DF938238910569F1DE
:1019A000B0F48133910509F46FC048F48932910590
:1019B00009F465C08A32910509F46BC08AC0853389
:1019C000910509F457C089339105B9F082C0833E6F
:1019D000910571F138F4803E9105B1F0823E910598
:1019E00011F177C0863E9105B9F1873E9105C9F1A5
:1019F000843E910509F06DC024C02091F20120FDC4
:101A000053C021FD51C065C08091F20180FD46C0E8
:101A10008091F30180FF48C08091F20184FD50C1A4
:101A200083EE90E04FC18091F20182FF3AC0F4CF83
:101A30008091F20182FD35C08091F30180FD34C0B8
:101A4000EBCF8091F30181FF35C08091F20184FDDD
:101A500037C187EE90E036C18091F20183FF27C045
:101A6000F4CF8091F20183FD22C08091F30181FDCA
:101A700021C0EBCF8091F20185FD1FC021C0809174
:101A8000F20185FD1DC019C08091F20186FD1BC0C9
:101A90001DC08091F20186FD19C015C089E390E058
:101AA00011C182EE90E00EC180EE90E00BC186EE97
:101AB00090E008C184EE90E005C189E290E002C1A7
:101AC00085E390E0FFC08AE290E0FCC081E390E013
:101AD000F9C0811531E5930708F069C0811540E52B
:101AE0009407F0F09C0174E0369527957A95E1F71C
:101AF000922F9370482F437021E030E002C0220FF4
:101B0000331F4A95E2F73C68392B982F9F709695C2
:101B1000969540E2949FC0011124822B932BD2C052
:101B2000883E910568F5803E910508F0CBC0883A63
:101B30009105B8F4853A910548F0855AE82FF0E010
:101B4000E55EFE4F808190E09064BCC081309105DD
:101B500009F4B3C008F4B4C08430910508F4B0C0EF
:101B6000B1C08F3B910508F0ABC0885AE82FF0E078
:101B7000EE0FFF1FE25EFE4F808191819464A2C050
:101B8000811520E2920758F4811531E0930708F09F
:101B900099C08D3E910508F493C0906593C081155E
:101BA00040E4940708F48CC09F70906A8BC0811544
:101BB00025E5920708F042C0811534E5930728F027
:101BC000982F8827846F906A7DC0811543E594071C
:101BD000B0F09C012370332741E050E002C0440F75
:101BE000551F2A95E2F7282F2695269580E2289FF3
:101BF00090011124CA01822B932B9A6863C081152E
:101C000022E5920728F4982F8827816F906A5AC09E
:101C10009C012370332741E050E002C0440F551F60
:101C20002A95E2F7282F2695269580E2289F900195
:101C30001124CA01822B932B9C6844C0EC018115AE
:101C400039E59307A8F48115984528F09C2F88273B
:101C5000806F906A37C0C11586E5D80788F58C2F4C
:101C60000E94AC0B8F7190E0982F882790622AC059
:101C700081152AE5920790F48C2F8F700E94AC0B8F
:101C800094E0D695C7959A95E1F7CF70D0E0DC2F18
:101C9000CC27D0699E01282BC90114C0905681150C
:101CA000904270F48D2F8F710E94AC0B282F2F71F2
:101CB000CE0199279062922B05C081E090E002C08E
:101CC00080E090E0DF91CF910895CF9384E090E0A1
:101CD0000E949223C82F82E290E00E9492232C2F30
:101CE00030E0A901582BCA01CF91089569EE7EEF2B
:101CF00080E090E00E94C42360E082E090E00E94D7
:101D0000A62360E083E090E00E94A6231092CF011A
:101D10001092D0011092D1011092D20160E084E0C3
:101D200090E00E94A62360E082E290E00E94A62359
:101D300060E085E090E00E94A62360E086E090E00D
:101D40000E94A6236FEF87E090E00E94A62340E068
:101D500050E0BA0188E090E00E94B82360E08DE096
:101D600090E00E94A62340E050E0BA0188E190E0B4
:101D70000E94B82360E087E190E00E94A62340E043
:101D800050E0BA018CE190E00E94B82360E070E07E
:101D900080E290E00E94C42340E050E0BA0188E174
:101DA00090E00E94B82340E050E0BA018FE090E05C
:101DB0000E94B82340E050E0BA0183E190E00C9427
:101DC000B8238091CE0181111092CE0108958095A3
:101DD0009091CD0189238093CD0108959091CD01FB
:101DE0008091CC01982B909383018091CE01882320
:101DF00089F0892B80938301E5E8F1E097E080E0AA
:101E0000915029F021912223D9F38F5FF9CF8111CD
:101E10000E94E10E48E050E064EC71E083E891E05C
:101E20000E946124892BA9F088E0E3E8F1E0A4ECAA
:101E3000B1E001900D928A95E1F7E0913602F091C0
:101E40003702309731F00280F381E02D83E891E092
:101E5000099408952091C301809582238093C30142
:101E6000982F977099F430E0482F082E000C550BEE
:101E70002417350759F09091F30192FD07C085951D
:101E8000859585950E946F221092C3010895CF9386
:101E9000C091F301C2FB992790F9981799F080FB44
:101EA000C2F9C093F3016091F20184E090E00E94D6
:101EB000A6236C2F82E290E00E94A62382E0CF91BD
:101EC0000C942A0FCF9108958091C20190919101B5
:101ED000891719F08F5F8770FBCF08950F931F93B9
:101EE000CF93DF938091900182958F7009F05DC050
:101EF00080918D01882309F458C08091C20110910E
:101F0000910160918B0170918C01C0918E01D091F3
:101F10008F0191E06F3F09F090E0292F06E08117D3
:101F200009F443C0209721F07F3F21F030E003C047
:101F300031E001C0322F90E030FD34C0089FF00145
:101F4000099FF00D1124DF01AE56BE4F11963C9152
:101F50001197371327C03C91361324C012963C9139
:101F6000129731111FC013964D915C9114974C1B21
:101F70005D0B483C5105B0F4809190018F708061F9
:101F800080939001E956FE4F80818F70806180833D
:101F90008BE891E00E94A804DF91CF911F910F91EF
:101FA0000C94640F01968770BACFDF91CF911F9187
:101FB0000F910895CF93DF93EC010E94B5212CE699
:101FC000829FC0011124FC0129E0D29FE00DF11D88
:101FD0001124EC0FF11DEE0FFF1FE852FF4F85910A
:101FE00094910E94CB0CDF91CF9108959F92AF9274
:101FF000BF92CF92DF92EF92FF920F931F93CF93F6
:10200000DF93CDB7DEB761970FB6F894DEBF0FBE92
:10201000CDBF8C0185E0F801DE011D9601900D9287
:102020008A95E1F7F801E28090918B0160918C0133
:1020300040918E0150918F014115510531F06F3F54
:1020400031F481E09F3F19F403C081E001C080E0DA
:10205000F82FF1709F2E80FD1AC1F8013081218187
:10206000C380D4808BE8A82E81E0B82EF0908D013B
:10207000F601E41BF50BFF2009F4C6C08091900126
:10208000E83CF10508F091C0482F407F09F050C0AE
:10209000621311C093130FC0FE2CE1100CC08F709F
:1020A000806180939001C5010E94A80480919001F5
:1020B000F801858329C1CD2831F02F3F31F481E02B
:1020C0003F3F19F403C081E001C080E080FD03C000
:1020D00081E08E2502C080E090E0F82FF170FF2EA5
:1020E00080FF1CC08091C2014091910156E084178D
:1020F00009F4E8C090E0589FF001599FF00D1124B9
:10210000EE56FE4F6181261306C06081631303C043
:102110006281E61203C001968770E9CFFE2CEE20A3
:1021200009F4F2C08091900181608093900149C0D0
:10213000621306C0931304C0E11002C0F80186C008
:10214000C8010E94BF22882351F1EE2041F1209165
:102150009001822F82958F7090E0029774F08091A9
:102160008B0190918C0198878F831986DB86CA86B4
:102170002C87CE0107960E94A80486E0F801ABE800
:10218000B1E001900D928A95E1F70E946E0F0AC0AE
:102190006217C9F0C8010E94BF2281111EC0C80188
:1021A0000E94A804FF24F394AFC0482F407F81F71A
:1021B0008BE891E00E94A80486E0F50111928A95CF
:1021C000E9F7F12CA1C09313E5CFE110E3CFF801BB
:1021D0008583C8010E94A80454C0EE2001F3209119
:1021E0009001822F82958F7090E0029734F2809157
:1021F0008B0190918C019A8389831B82DD82CC8232
:102200002E83CE010196B7CFE83CF105D0F5FE2C28
:10221000EE2029F2621327C0931325C0209190016C
:1022200020FD18C0822F82958F70482F50E04115F5
:10223000510581F0F80125834F30510541F08F5F42
:10224000982F9295907F822F8F70892B8583C8015C
:102250000E94A80486E0F801ABE8B1E001900D927D
:102260008A95E1F751C0C8010E94BF22811185CF34
:1022700080919001816080939001C8010E94A80420
:1022800043C086E0F50111928A95E9F73DC0EE2042
:1022900009F485CFC8010E94BF22F82E882309F4D3
:1022A0007ECF86E0F801ABE8B1E001900D928A950F
:1022B000E1F780918B0190918C010E94DA0F0E94CE
:1022C0006E0F22C03D872E878D859E850E94DA0F76
:1022D000292F22952F70223028F49F7039F0811118
:1022E00005C00BC0243028F49F7049F4805E88300C
:1022F00020F0C8010E94A8049F2CF92C05C0F80109
:102300009581907F99F7F9CF8F2D61960FB6F8944C
:10231000DEBF0FBECDBFDF91CF911F910F91FF9018
:10232000EF90DF90CF90BF90AF909F900895CF93A4
:10233000DF93CDB7DEB760970FB6F894DEBF0FBE60
:10234000CDBF84B7877F84BF0FB6F894A8958091DE
:102350006000886180936000109260000FBE90E082
:1023600080E80FB6F89480936100909361000FBEEF
:1023700085B7806885BF85B7806885BF8AEA9BE09E
:1023800090938101809380010E94E91C0E94081DA6
:102390008091E20084608093E200789480914F0203
:1023A0008823A1F01091E9001F709091EC00892F13
:1023B000817090FD80E8182B1092E9008091E80070
:1023C00083FD0E94D8191F701093E90082E084BD3C
:1023D00093E095BD9AEF97BD80936E000CE411E0F9
:1023E000F8E5EF2EF1E0FF2ED8018D918D018F3FA2
:1023F00011F00E94EF0BE016F106B1F708E511E0CD
:10240000E1E6EE2EE1E0FE2EF80181918F018F3F93
:1024100011F00E94EF0BE016F106B1F788E1E7EF4B
:10242000F1E0DF01282F1D922A95E9F7E6EDF1E0B2
:10243000DF011D928A95E9F76E9A229A80E090E07A
:102440000E94A023893E9E4F11F00E94760E82E0EA
:1024500090E00E94922380930F020E94650E909359
:10246000F3018093F2010E94060CEFEFF6E721E002
:10247000E150F0402040E1F700C000000E94060C4F
:102480008091F70180FF08C06FEF7FEF80E090E060
:102490000E94C4230E94431783E090E00E9492238D
:1024A000682F70E080E090E00E94B522279A2F9874
:1024B0008AE08093800089E1809381008FEF9FEF15
:1024C00090938700809386000E9466190E94661987
:1024D0008091F401811136C080E090E00E94A02339
:1024E000893E9E4F21F00E94760E0E94B01E88E029
:1024F00090E00E949A2360932B0270932C028093A9
:102500002D0290932E026E7F71F40E94B01E88E01F
:1025100090E00E949A2360932B0270932C02809388
:102520002D0290932E020E94691E10926D028091DE
:102530002B0280FF04C060E086950E940E2081E09F
:102540008093F40180E091E090933702809336020B
:1025500058E1E52EF12C60E4B62E7FE0C72E72E044
:10256000D72E80914F02853009F07CC09924939436
:1025700000E112E180914F02853009F05AC080914C
:102580004F02843009F443C080E00E94AE1880E01E
:102590000E949A0410926D028091F601811116C07A
:1025A0009092F60180912B02982F91709093F501F3
:1025B0008E7F80932B024FEF80E792E04150804066
:1025C0009040E1F700C000000E94561E10923A02AF
:1025D0000FB6F894A895E09260000FBEB09260002C
:1025E00083B7817F846083BF83B7816083BF789422
:1025F000889583B78E7F83BF0FB6F894A895809196
:102600006000886180936000109260000FBE80912E
:102610004E02882309F4AECF0E94060CE7EFF1E0EA
:1026200081919191892B09F0F8C1CE16DF06C1F78F
:10263000A1CF0E94DF220E9466190E9417180E94F3
:102640009A041092F6018091F501882349F0809157
:102650002B02816080932B0260E086950E940E2001
:102660000E94401E0E94060C882359F08FB7F894F0
:1026700040913B0250913C0260913D0270913E02BC
:102680008FBFA7EFB1E0E0E1F2E000E010E0702FD3
:102690002D913D918191919182279327009779F116
:1026A00060E088248394912CAC0148215921452B6A
:1026B00009F16F8378872821392181E0232B09F4E0
:1026C00080E089870E949C178160782F9B878A878A
:1026D0004F81588569858B850E94F203000F111F79
:1026E000F801E05FFD4F80819181882699269182D3
:1026F00080821AC06F5F880C991C6930A9F60F5F41
:102700001F4F0C30110519F68FEF8C878D871E86B1
:102710000E949C178160782F988B8F874C855D85F0
:102720006E8588890E94F20380916D02882309F4E6
:1027300085C080916C02E0912B02E695E81BE09346
:102740006802823059F4F0E0ED5BFB4FE4910E2F0C
:1027500010E07AE4872E76E1972E4BC0863059F44C
:10276000F0E0E05CFB4FE4910E2F10E06AE3862E70
:1027700066E1962E3EC0893061F4E695F0E0E35CB8
:10278000FB4FE4910E2F10E05AEE852E55E1952E69
:1027900030C08F3059F4F0E0E65CFB4FE4910E2F2F
:1027A00010E044ED842E45E1942E23C08231A1F047
:1027B0008D3149F4E8E3F4E0059114913AEF832E6A
:1027C00035E1932E16C08E3171F404EF11E020EB49
:1027D000822E25E1922E0DC008E210E09EEB892E9C
:1027E00095E1992E06C000ED17E081E3882E85E182
:1027F000982E80916902882361F0109269020E94EC
:102800009C17909367028093660210926B0210925D
:102810006A020E949C17E0916602F09167028E1B8B
:102820009F0B8F3F9F4750F40E0F1F1F109367029F
:102830000093660286E692E0F401099586E0E0E600
:10284000F2E0DE01119601900D928A95E1F78090F9
:1028500062029090630200916402109165021092EE
:10286000620210926302109264021092650281105B
:1028700003C0992009F451C080915E0290915F02DB
:102880000E948D179C0190915A02992309F4DBC094
:102890002531310508F441C09F3F19F09F5F9093A7
:1028A0005A02882061F00E941F21181414F09FEF33
:1028B00001C091E0899F802D1124809362029920AC
:1028C00061F00E941F21191414F09FEF01C091E0E4
:1028D000899F802D112480936302309162023323FB
:1028E000E1F0209163022223C1F045EB3403C001E3
:1028F0001124992319F09093620203C081E0809320
:10290000620235EB2303C0011124992319F090933F
:10291000630203C081E080936302011103C01123AD
:1029200009F451C080915C0290915D020E948D1764
:102930009C0190915902992309F48AC021353105EF
:1029400008F441C09F3F19F09F5F90935902002304
:1029500061F00E94FD20101614F09FEF01C091E07D
:10296000899F802D112480936402112361F00E94BD
:10297000FD20111614F09FEF01C091E0899F802D7A
:10298000112480936502309164023323E1F0209199
:1029900065022223C1F045EB3403C00111249923C1
:1029A00019F09093640203C081E08093640235EBD8
:1029B0002303C0011124992319F09093650203C0E9
:1029C00081E0809365028091620281110BC0809149
:1029D0006302811107C080916402811103C080915C
:1029E000650281110E945C208B829C820D831E8374
:1029F00086E0FE013196A0E6B2E001900D928A9544
:102A0000E1F70E94171890912802891709F4A9CDBF
:102A1000809328020E949A04A4CD09BD19BD09B46F
:102A200000FEFDCF8091D8008F7D8093D8008091EB
:102A3000E00082608093E0008091E00081FDFCCFA7
:102A40000E94DF2297CD2B30310508F027CF65CFCC
:102A50002B30310508F078CFB6CF0895809144022D
:102A60000895089580933F0270934102609340025D
:102A700080914F02843001F582E08093E9008FEF6E
:102A80009091E800815095FD06C095ED9A95F1F77B
:102A900000008111F5CF8091E80085FF0DC040E076
:102AA00050E063E070E08FE392E00E94AC19809107
:102AB000E8008E778093E8000895BC0184E00C94D0
:102AC0003215BC0183E00C94321522E02093E9001A
:102AD0002FEF3091E800215035FD06C035ED3A95D5
:102AE000F1F700002111F5CF2091E80025FF0BC080
:102AF00040E050E066E070E00E94AC198091E80090
:102B00008E778093E8000895CF93DF9321E02093A0
:102B1000E9002FEF3091E800215035FD06C035ED7A
:102B20003A95F1F700002111F5CF2091E80025FF3B
:102B300014C0EC0140E050E068E070E00E94AC1985
:102B40008091E8008E778093E80088E0FE01A5E49C
:102B5000B2E001900D928A95E1F7DF91CF9108954F
:102B6000CF93DF93EC010E94561E8C8190E001967A
:102B7000817099278C83DF91CF910895CF93DF9354
:102B8000EC010E94561E8C81811102C091E003C0AD
:102B9000803219F49FEF90930E0190910E01890FEE
:102BA0008C83DF91CF9108950E94561E80910C0175
:102BB00090912902980F9093290220910D01280FDE
:102BC00020930D01121614F49F3F1CF08195809301
:102BD0000C010895CF93DF93EC010E94561E9A8159
:102BE0008C8190FF02C08F5F01C081508C83DF9188
:102BF000CF9108950F931F93CF93DF9300D01F922F
:102C0000CDB7DEB78C0180912A0281110AC09E01E6
:102C10002F5F3F4F4FEF6FEF0E94BF1E8A8180935F
:102C20002A02F8018481813051F028F0823061F469
:102C300040912A020AC080912A0240E007C06091B8
:102C40002A0240E080E003C040E080E060E00E94B3
:102C5000631EF801848190E0019663E070E00E94B9
:102C6000FE2384830F900F900F90DF91CF911F91DF
:102C70000F910895CF93DF93EC01EBE2F2E04381F3
:102C800062818C810E94551F8C818F5F8C83DF91C4
:102C9000CF910895CF93DF93EC01EC81F0E0E95BF5
:102CA000FB4F4491EBE2F2E0628181810E94551F6B
:102CB0008C818F5F8C83DF91CF9108952091E40008
:102CC0003091E50095E64091EC00842F817040FF43
:102CD00023C08091E80080FD1DC080914F028823B1
:102CE00099F0853099F08091EB0085FD11C04091FD
:102CF000E4005091E5002417350729F3915011F0B5
:102D00009A01E1CF84E0089582E0089583E0089578
:102D100081E0089580E008954091E80042FFDDCF12
:102D200008958091510287FF11C08091E80082FDD3
:102D300005C080914F028111F8CF11C08091E80049
:102D40008B770BC080914F02882349F08091E80077
:102D500080FFF8CF8091E8008E778093E800089597
:102D6000982F973068F59093E900981739F0709193
:102D7000EC002091ED005091F00003C0242F762F3D
:102D800050E021FD02C09F5FECCF3091EB003E7F11
:102D90003093EB003091ED003D7F3093ED003091AA
:102DA000EB0031603093EB007093EC002093ED006A
:102DB0005093F0002091EE0027FDE5CF80E00895CC
:102DC0008F708093E90081E008952091570230913F
:102DD00058022617370748F06115710539F420911C
:102DE000E8002E772093E80001C0B901FC0120E043
:102DF0006115710579F180914F028823F1F18530D9
:102E0000F1F18091E80083FD3CC08091E80082FDF3
:102E10002EC08091E80080FFEBCF2091F3008091DD
:102E2000F20090E0922B6115710551F08830910508
:102E300038F421912093F100615071090196F3CF8C
:102E400021E0089709F020E08091E8008E778093D8
:102E5000E800CECF2111CFCF0AC080914F02882346
:102E600061F0853061F08091E80083FD0AC08091B7
:102E7000E80082FFF2CF80E0089582E0089583E0C9
:102E8000089581E0089581E08093E00080E28093DE
:102E9000D8001092C9008FE19EE40197F1F700C0BD
:102EA000000087E090EBDC018093B4029093B502C0
:102EB000A093B602B093B7029CE088E10FB6F894F5
:102EC000A895809360000FBE90936000FFCF789428
:102ED0001F920F920FB60F9211248F939F93AF936F
:102EE000BF9380913B0290913C02A0913D02B09132
:102EF0003E020196A11DB11D80933B0290933C02BE
:102F0000A0933D02B0933E02BF91AF919F918F91EC
:102F10000F900FBE0F901F9018959C014FB7F8941B
:102F200080913B0290913C02A0913D02B0913E0203
:102F30004FBF821B930B08952FB7F89480913B02EB
:102F400090913C02A0913D02B0913E022FBF0895A6
:102F50001F920F920FB60F9211248F939F93AF93EE
:102F6000BF9380913A02811113C080913B029091EE
:102F70003C02A0913D02B0913E024196A11DB11DBF
:102F800080933B0290933C02A0933D02B0933E029B
:102F9000BF91AF919F918F910F900FBE0F901F9097
:102FA00018959C01FC0132969FEF80E041914617F5
:102FB00089F09F3F19F4411101C0982F8F5F86302F
:102FC000A9F79F3F39F0F901E90FF11D97FDFA9537
:102FD00062830895089520913802309139022817AC
:102FE000390771F09093390280933802E0913602EC
:102FF000F0913702309721F00084F185E02D09949B
:10300000089520913402309135022817390771F064
:103010009093350280933402E0913602F0913702AA
:10302000309721F00680F781E02D09940895E09112
:103030003602F0913702309721F00190F081E02DB7
:10304000099480E00895EF92FF920F93CF93DF935E
:10305000C42FD22FFC0182818823D1F04093330208
:103060000E949C17909332028093310280E28C0F71
:10307000883008F06DC0C77081E001C0880FCA9524
:10308000EAF7DF91CF910F91FF90EF900C94F1222E
:103090008091330248134BC08091310290913202EB
:1030A0000E948D17883C910508F041C0CD17C9F0EA
:1030B00080E28C0F883040F4C77081E001C0880F37
:1030C000CA95EAF70E94EA2280E28D0F883048F420
:1030D00081E09D2F977001C0880F9A95EAF70E94B2
:1030E000F122093319F0E12CF12C03C080E5E82E20
:1030F000F12C802F0E943323E114F10451F08FE969
:103100009FE00197F1F700C0000091E0E91AF10893
:10311000F3CF802F0E94FB2280E28D0F8830C0F415
:10312000D77081E001C0880FDA95EAF70AC080E223
:103130008C0F883068F4C77081E001C0880FCA9591
:10314000EAF7DF91CF910F91FF90EF900C94EA2274
:10315000DF91CF910F91FF90EF9008958F929F9202
:10316000AF92BF92CF92DF92EF92FF920F931F9395
:10317000CF93DF93863048F4811108C0909180008E
:10318000977F909380002F9806C085E090918000F3
:10319000986090938000A0918600B0918700282FBE
:1031A00030E00E943A2425E030E040E050E00E9408
:1031B00012240027122F232F342F012F122F232FF9
:1031C000332780918600909187006CE070E00E9428
:1031D000EA236017710730F0C80169E070E00E94CF
:1031E000EA235EC08091860090918700E09086007F
:1031F000F0908700E0918600F0918700C6E0D0E073
:10320000BE010E94EA23060F171F211D311D480130
:10321000590185E0880C991CAA1CBB1C8A95D1F722
:10322000C701BE010E94EA236F01E12CF12CA70126
:103230009601260F371F411D511DC501B4010E9483
:10324000122469017A01E0918600F0918700CA0199
:10325000B9010E94DA239B01AC01DF010E944924DD
:103260009B01AC01C701B6010E94DA23DC01CB014E
:103270002FE0B695A795979587952A95D1F7009158
:1032800086001091870020E030E0081719072A0710
:103290003B0728F46091860070918700CB01BC0148
:1032A00070938D0060938C00DF91CF911F910F91EF
:1032B000FF90EF90DF90CF90BF90AF909F908F9056
:1032C0000895682F86E090E00C94A62380E090E0BB
:1032D0000E94A023893E9E4F51F00E94760E80915D
:1032E000300284708962809330020E94611986E006
:1032F00090E00E94922380933002282F26952695F5
:10330000269530E02630310524F08770886280935E
:1033100030028091300280FF04C0869586958695A4
:1033200001C080E00C94AE1890912B0290FF04C075
:103330009695981740F003C0811105C090E096174C
:1033400010F40C94522061E00C940E20882311F0AC
:10335000FA0101C0FB010994EF92FF920F931F93B2
:10336000CF93DF937C018B010E945E16811119C0FF
:10337000E70101151105A1F08091E80085FD0AC063
:103380008091E8008E778093E8000E945E16882383
:1033900081F307C089918093F10001501109E9CFB1
:1033A00080E0DF91CF911F910F91FF90EF900895F2
:1033B0001F93CF93DF93CDB7DEB7AA970FB6F894DC
:1033C000DEBF0FBECDBFE1E5F2E089E592E02091DE
:1033D000F10021938E179F07D1F78091520283301D
:1033E00009F461C030F4813071F0823009F49BC07F
:1033F000B2C08A3009F487C08B3009F46CC08930C0
:1034000009F0A9C020C080915102813A09F0A3C0FF
:103410008091E800877F8093E80080915502909129
:103420005602892B21F468E085E492E003C060E055
:1034300080E090E070E00E94E5168091E8008B77D4
:103440008093E80088C080915102813209F083C0E6
:103450008091550290915602029708F07CC08091AD
:10346000E800877F8093E8008091E80082FD05C036
:1034700080914F028111F8CF6EC02091F3008091AE
:10348000F20090E0922B029731F48091F1008130AC
:1034900011F0863021F48091F100809344028091F4
:1034A000E8008B7754C080915102813A09F053C0F3
:1034B0008091550290915602892B09F04CC0809161
:1034C000E800877F8093E8008091E80080FFFCCFD0
:1034D00080910F0137C0809151028132E1F58091D6
:1034E000550290915602892BB1F58091E800877FB3
:1034F0008093E8000E9491168091530280930F01FF
:103500000E94DF2228C080915102813221F58091F2
:10351000E800877F8093E8000E9491168091540212
:103520008093430218C080915102813AA1F48091A6
:10353000E800877F8093E8008091E80080FFFCCF5F
:10354000809143028093F1008091E8008E77809310
:10355000E8000E9491168091E80083FFCEC180911F
:10356000510290915202492F50E04A30510508F023
:10357000C4C1FA01EE59FF4F0C943424803821F075
:10358000823809F0BAC108C080914D0290914E0274
:10359000992389F082600FC0809155028F70873027
:1035A00008F0ABC18093E9008091EB0085FB882790
:1035B00080F91092E9009091E800977F9093E800DD
:1035C0008093F1001092F10065C1282F2D7F09F042
:1035D00094C1882319F0823061F08FC18091530229
:1035E000813009F08AC1933009F080E080934E0267
:1035F0002EC08091530281112AC0809155028F7094
:103600002FEF280F263008F078C18093E900209131
:10361000EB0020FF1CC0933021F48091EB0080620E
:1036200014C09091EB0090619093EB0021E030E0AA
:10363000A90102C0440F551F8A95E2F74093EA00A2
:103640001092EA008091EB0088608093EB0010926A
:10365000E9008091E800877F20C181114EC110915F
:1036600053021F778091E3008078812B8093E300E1
:103670008091E800877F8093E8000E9491168091F6
:10368000E80080FFFCCF8091E30080688093E30036
:10369000111102C082E001C083E080934F022DC16E
:1036A0008058823008F029C18091530290915402D1
:1036B0008C3D53E0950779F583E08A838AE289831C
:1036C0004FB7F894DE01139620E03EE051E2E32F7D
:1036D000F0E050935700E49120FF03C0E295EF70B3
:1036E0003F5FEF708E2F90E0EA3010F0C79601C078
:1036F000C0968D939D932F5F243149F74FBF8091E2
:10370000E800877F8093E8006AE270E0CE010196CE
:103710000E94E516AEC04091550250915602292FE5
:10372000332723303105A9F068F42130310509F43D
:10373000F3C02230310509F0E0C08BE390E0E2E015
:10374000F6E044C02132310521F12232310571F118
:10375000D4C0992781309105A1F058F0029709F063
:10376000CCC0EFE4F6E0E4918E2F90E0EFE4F6E0D9
:103770002AC0E7E6F6E0E4918E2F90E0E7E6F6E077
:1037800022C0EDE5F6E0E4918E2F90E0EDE5F6E065
:103790001AC04115510509F4C4C04130510509F062
:1037A000ACC089E090E0EDE2F6E010C041155105B3
:1037B00009F4BCC04130510509F09FC08BE790E08F
:1037C000E7E4F5E003C0009709F497C02091E80012
:1037D000277F2093E80020915702309158028217EA
:1037E000930708F49C0140E02115310589F180918F
:1037F0004F02882309F43DC08530D9F18091E8005B
:1038000083FD37C08091E80082FD2FC08091E800E1
:1038100080FFEACF4091F3008091F20090E0942B7A
:103820002115310559F08830910540F444914093B9
:10383000F1003196215031090196F2CF41E008970D
:1038400009F040E08091E8008E778093E800CCCFCB
:103850004111CDCF0AC080914F02882351F08530AD
:1038600041F08091E80083FD04C08091E80082FF70
:10387000F2CF8091E8008B778093E8003EC08038DB
:10388000E1F58091E800877F8093E8008091500205
:103890008093F1008091E8008E778093E8000E9489
:1038A00091162BC0811129C080915302909154022E
:1038B0009927029714F58091E800877F8093E800AC
:1038C00010915302109350020E949116111106C0DC
:1038D0008091E30087FD02C081E001C084E0809315
:1038E0004F0242E061EC81E00E94B01642E261ECDE
:1038F00082E00E94B01680914F028091E80083FF21
:103900001AC08091E800877F8093E8008091EB00E7
:1039100080628093EB000FC082E190E0EDE3F6E07F
:1039200055CF89E090E0E4E1F6E050CF80E490E00C
:10393000E2ECF5E04BCFAA960FB6F894DEBF0FBECF
:10394000CDBFDF91CF911F9108951F920F920FB6B7
:103950000F9211242F933F934F935F936F937F9315
:103960008F939F93AF93BF93CF93DF93EF93FF9387
:10397000C091E900CF708091EC00D82FD17080FD0C
:10398000D0E81092E9008091F000877F8093F000EA
:1039900078940E94D8191092E9008091F000886014
:1039A0008093F000CD2BCF70C093E900FF91EF9191
:1039B000DF91CF91BF91AF919F918F917F916F9147
:1039C0005F914F913F912F910F900FBE0F901F90DD
:1039D0001895E8EDF0E080818E7F80831092E20000
:1039E0001092DA001092E100A0EEB0E08C918160BC
:1039F0008C9380818F77808319BCA7EDB0E08C9188
:103A00008E7F8C9380818F7E8083109242020895F6
:103A1000CF92DF92EF92FF920F931F93CF93DF939A
:103A2000C8EDD0E088818F7E8883E7EDF0E080816B
:103A30008160808384E082BF81E08093420288813C
:103A40008E7F888302EE10E0F80110821092DA0077
:103A500081EEC82ED12CF601108288818F77888361
:103A600088818068888388818F7D888319BC1092C3
:103A70004F021092500210924E0210924D0290EEA0
:103A8000E92EF12CF70180818B7F80838881816012
:103A9000888342E060E080E00E94B016F6018081F9
:103AA0008E7F8083F801808181608083808188603F
:103AB0008083F70180818E7F808388818061888305
:103AC000DF91CF911F910F91FF90EF90DF90CF90FA
:103AD00008951F920F920FB60F9211242F933F93C8
:103AE0004F935F936F937F938F939F93AF93BF9306
:103AF000EF93FF938091E10082FF09C08091E20083
:103B000082FF05C08091E1008B7F8093E10080916E
:103B1000DA0080FF2AC08091D80080FF26C0809103
:103B2000DA008E7F8093DA008091D90080FF18C080
:103B300080E189BD82E189BD09B400FEFDCF81E04D
:103B400080934F028091420281110FC00E94E91CB4
:103B50000E94081D8091E20084608093E20005C00D
:103B600019BC10924F02109242028091E10080FF36
:103B700017C08091E20080FF13C08091E2008E7F29
:103B80008093E2008091E20080618093E200809166
:103B9000D80080628093D80019BC85E080934F02E2
:103BA0008091E10084FF30C08091E20084FF2CC04E
:103BB00080E189BD82E189BD09B400FEFDCF80911D
:103BC000D8008F7D8093D8008091E1008F7E809314
:103BD000E1008091E2008F7E8093E2008091E2001C
:103BE00081608093E20080915002882311F084E08C
:103BF00007C08091E30087FD02C081E001C083E03F
:103C000080934F0280914F028091E10083FF27C093
:103C10008091E20083FF23C08091E100877F809341
:103C2000E10082E080934F02109250028091E10007
:103C30008E7F8093E1008091E2008E7F8093E2008E
:103C40008091E20080618093E20042E060E080E0E9
:103C50000E94B0168091F00088608093F000FF9180
:103C6000EF91BF91AF919F918F917F916F915F91F4
:103C70004F913F912F910F900FBE0F901F9018956D
:103C800060912B02669570E04BE050E080E191E09E
:103C90000E945424892B19F481E080936D020E94C4
:103CA0009C1790936702809366020895239A85B1CA
:103CB00085B18FB7F8948FBF8FE594E00197F1F746
:103CC00000C00000089580912B0280FD0C94561EC8
:103CD000089580912B02282F269530E0211531057B
:103CE00019F48170826005C02F31310524F0817094
:103CF0008C6380932B020895CF92DF92EF92FF9214
:103D00006B017C010E94691EB701A60188E090E06A
:103D1000FF90EF90DF90CF900C94B82380912F020A
:103D2000882319F0815080932F0260912B027091AB
:103D30002C0280912D0290912E020C947C1E809179
:103D40002F02833018F48F5F80932F0260912B0233
:103D500070912C0280912D0290912E020C947C1E69
:103D6000EBE2F2E083E0808311828FEF8283838332
:103D7000148260817181828193810C947C1EAF9248
:103D8000BF92CF92DF92EF92FF920F931F93CF9348
:103D9000DF93E82EF62EE901E42FF0E0611106C072
:103DA000E559F94FE4914E2F2E2F71C0062F10E0E8
:103DB000E559F94F4491F42FC42ED12C26E0829F6F
:103DC000C00111242FEF30E0B9010E94EA235BEA21
:103DD0005603C001579F900D11248E0D911D8E0D1D
:103DE000911D582F550F580FD901A01BB10BAC9D39
:103DF000C001AD9D900DBC9D900D1124E92FF59E45
:103E0000D0011124AB2FBB277901EA1AFB0AEC9CE5
:103E1000D001ED9CB00DFC9CB00D11245901A51AE8
:103E2000B108A09E7001A19EF00CB09EF00C112470
:103E3000EF2CFF242E193F092C9D80012D9D100D84
:103E40003C9D100D1124212F6230710591F048F432
:103E500061157105E1F061307105B9F4242F4B2F24
:103E600016C06430710569F040F06630710579F074
:103E70000CC0242F492FE12F0AC0492FEF2F2B2FE1
:103E800006C0292FE42F412F02C0292FEB2F498391
:103E90002883EA83DF91CF911F910F91FF90EF90DC
:103EA000DF90CF90BF90AF900895CF93DF9300D075
:103EB0001F92CDB7DEB790912B0290FF0AC09E01F2
:103EC0002F5F3F4F0E94BF1E4B8169818A810E94F4
:103ED000631E0F900F900F90DF91CF910895EF9296
:103EE000FF920F931F93CF93DF9300D01F92CDB714
:103EF000DEB7082FF62E142FE22E90912B0290FFA2
:103F000041C0E92FE695AE2FB0E0AF59BE4F8C917E
:103F100080936C029E7F923061F49E012F5F3F4F31
:103F2000802F0E94BF1E4B8169818A810E94631E7F
:103F300017C0823019F410912E0212C0863019F485
:103F400000912C020DC08930D9F3833149F4E3513B
:103F5000E695F0E0E559F84F859194910E94561E40
:103F600000932C02F0922D0210932E02EE2051F0BD
:103F700060912B0270912C0280912D0290912E0263
:103F80000E947C1E0F900F900F90DF91CF911F9198
:103F90000F91FF90EF900895EBE2F2E0438128E06B
:103FA000421B08F440E021E0628181810C946F1F84
:103FB000EBE2F2E0438128E0420F08F44FEF21E00A
:103FC000628181810C946F1FEBE2F2E0628128E054
:103FD000621B08F460E021E0438181810C946F1F33
:103FE000EBE2F2E0628128E0620F08F46FEF21E07B
:103FF000438181810C946F1FEBE2F2E0818121E02B
:104000004381628188500C946F1FEBE2F2E0818162
:1040100021E043816281885F0C946F1F90912B0295
:1040200090FF36C09170811102C0926006C08F313E
:1040300010F09C6302C0880F982B90932B0266238C
:1040400051F060912B0270912C0280912D02909181
:104050002E020E947C1E60912B02669570E04BE060
:1040600050E080E191E00E945424892B19F01092D5
:104070006D0202C00E94401E81E08093690220E030
:1040800040912E0260912D0280912C020C946F1FA2
:10409000089580912B028695815009F48EE161E0AC
:1040A0000C940E2080912B0286958F5F8F3108F043
:1040B00081E061E00C940E200E949C172091620226
:1040C000211104C020916302222321F090935F020A
:1040D00080935E0220916402211104C02091650248
:1040E000222321F090935D0280935C02E0913602DE
:1040F000F0913702309749F082E0809360020480AB
:10410000F581E02D80E692E0099408958D3E39F422
:104110009091630297FF35C01092630259C08E3EA2
:1041200029F4909163021916BCF32BC0909162029E
:104130008F3E29F497FF25C01092620249C0803F4C
:1041400019F41916CCF31DC090916402893F29F42B
:104150001916BCF4109264023BC08A3F19F497FF11
:1041600010C0F8CF8B3F39F49091650297FF09C0DA
:10417000109265022DC08C3F21F4909165021916B2
:10418000BCF39FE0980F983080F421E030E0A90163
:1041900002C0440F551F9A95E2F7CA01809590918D
:1041A000610289238093610213C08D3F21F48091C5
:1041B0005B028E7F0BC08E3F21F480915B028D7F6E
:1041C00005C08F3F29F480915B028B7F80935B0257
:1041D00080916202811106C080916302811102C048
:1041E00010925A0280916402811106C0809165028A
:1041F000811102C010925902089580915B0280FDE6
:1042000016C081FD16C082FD18C080915902882316
:1042100091F0883290F428E0829FC001112468E276
:1042200070E00E94FE23862F672B29F007C082E0F2
:10423000089584E0089581E0089588E008958091CC
:104240005B0280FD14C081FD14C082FD16C0809108
:104250005A02882381F08E3180F420E5829FC001CC
:1042600011246EE170E00E94FE23862F089584E100
:10427000089588E2089588E0089580E508958D3EC8
:1042800021F40E941F21819504C08E3E29F40E94D2
:104290001F218093630208958F3E21F40E941F2105
:1042A000819504C0803F29F40E941F2180936202FF
:1042B0000895893F19F40E94FD2005C08A3F31F41A
:1042C0000E94FD2081958093640208958B3F21F424
:1042D0000E94FD20819504C08C3F29F40E94FD209E
:1042E0008093650208959FE0980F983078F421E05C
:1042F00030E0A90102C0440F551F9A95E2F7CA01A8
:1043000090916102892B8093610208958D3F21F481
:1043100080915B0281600BC08E3F21F480915B0233
:10432000826005C08F3F29F480915B028460809396
:104330005B02089580E090E00E94011880E090E028
:104340000E94EB171092CC010E94EE0EE0E6F2E024
:1043500086E0DF011D928A95E9F710925A021092C9
:10436000590210925B020C945C208F929F92AF9244
:10437000BF92DF92EF92FF920F931F93CF93DF9341
:104380008090EE019090EF01A090F001B090F101CB
:104390004091CF015091D0016091D1017091D20133
:1043A000842A952AA62AB72ACFE1D0E029E0929F55
:1043B000700111249CE6D92E082F10E0D501C4010C
:1043C0000C2E04C0B695A795979587950A94D2F7B9
:1043D00080FD04C0219790F780E014C0DC9EF001BE
:1043E000DD9EF00D1124EE0DFF1DE00FF11FEE0F0D
:1043F000FF1FE852FF4F859194910E94CB0C0197CB
:1044000049F38C2FDF91CF911F910F91FF90EF9087
:10441000DF90BF90AF909F908F90089529E0929F7A
:10442000800D1124682F669566956695982F977074
:1044300085E0689FB001112440E050E080E0FB017E
:10444000E40FF51FE259FD4F208130E0092E02C034
:10445000369527950A94E2F721703327042E01C080
:10446000220F0A94EAF7822B4F5F5F4F45305105C8
:1044700031F7089529E0929F800D1124E82FE695E9
:10448000E695E695877051E001C0550F8A95EAF7E9
:1044900085E0E89FF0011124E259FD4F20E030E073
:1044A00070E04081CB01022E02C0969587950A9458
:1044B000E2F78170819584278523842781932F5F7C
:1044C0003F4F2530310569F708956093EE017093F1
:1044D000EF018093F0019093F1010C949A210F93D6
:1044E0001F9341E050E060E070E004C0440F551FAE
:1044F000661F771F8A95D2F7409550956095709505
:104500008091EE019091EF01A091F001B091F10145
:104510008A019B01082319232A233B23C901B801DF
:104520001F910F910C9465220F931F9341E050E06F
:1045300060E070E004C0440F551F661F771F8A9526
:10454000D2F78091EE019091EF01A091F001B0912E
:10455000F1018A019B01082B192B2A2B3B2BC90146
:10456000B8011F910F910C9465226093CF01709355
:10457000D0018093D1019093D2010C949A21FC0137
:10458000808191810E94DA0F92959F70963079F028
:1045900010F4925001C09A50923068F4803F69F054
:1045A00018F4883E40F409C0843F29F406C0883ED0
:1045B00020F0813F11F080E0089581E0089510928D
:1045C000CD0186E0E5E8F1E0DF011D928A95E9F78B
:1045D0000C949A21882321F00E94E70E0C94EE0E91
:1045E0000895882339F09091CD01892B8093CD01D6
:1045F0000C94EE0E08958823A9F19CEF980F913A40
:1046000060F4E3E8F1E09281891301C012823196EF
:1046100091E0E938F907B9F70DC090E2980F9830AA
:1046200058F4877091E001C0990F8A95EAF7892FB5
:104630000E94E70E0C94EE0E9BE5980F933020F449
:1046400080E090E00C94011898E5980F973120F4E1
:1046500080E090E00C94EB178D3E20F00E948620C5
:104660000C945C200895CF93882309F459C0C82F77
:104670008CEF8C0F813AF8F4E5E8F1E08BE891E0FB
:104680002191C21721F08E179F07D1F70EC0E3E8E2
:10469000F1E089E891E02281C21301C012823196D3
:1046A0008E179F07C1F70E94EE0E6C2F83E891E0F2
:1046B0000E94D11710C080E28C0F883078F4C77048
:1046C00081E090E001C0880FCA95EAF79091CD0192
:1046D000892B8093CD01CF910C94EE0EEBE5EC0F7E
:1046E000E33040F4F0E0E55EFE4F808190E0CF9152
:1046F0000C940118E8E5EC0FE73150F4F0E0EE0F10
:10470000FF1FE25EFE4F80819181CF910C94EB17E9
:10471000CD3E30F08C2F0E943F21CF910C945C2035
:10472000CF910895F999FECF92BD81BDF89A99274E
:1047300080B50895A6E1B0E044E050E00C94CC23AD
:10474000A8E1B0E042E050E00C94CC23262FF99988
:10475000FECF92BD81BDF89A019700B4021639F0E0
:104760001FBA20BD0FB6F894FA9AF99A0FBE0895B1
:104770000396272F0E94A7230E94A623252F0E947D
:10478000A723242F0C94A7230196272F0E94A72349
:104790000C94A623DC01CB01FC01F999FECF06C0E5
:1047A000F2BDE1BDF89A319600B40D9241505040EF
:1047B000B8F70895DB018F939F930E944924BF911E
:1047C000AF91A29F800D911DA39F900DB29F900D60
:1047D00011240895AA1BBB1B51E107C0AA1FBB1FD0
:1047E000A617B70710F0A61BB70B881F991F5A957D
:1047F000A9F780959095BC01CD01089597FB072EF0
:1048000016F4009407D077FD09D00E94EA2307FC34
:1048100005D03EF4909581959F4F089570956195D0
:104820007F4F0895A1E21A2EAA1BBB1BFD010DC0EC
:10483000AA1FBB1FEE1FFF1FA217B307E407F50750
:1048400020F0A21BB30BE40BF50B661F771F881F2C
:10485000991F1A9469F760957095809590959B01C2
:10486000AC01BD01CF010895EE0FFF1F0590F4913B
:10487000E02D0994A29FB001B39FC001A39F700DCA
:10488000811D1124911DB29F700D811D1124911D58
:1048900008950E943A24A59F900DB49F900DA49F67
:1048A000800D911D11240895FC014150504030F0BD
:1048B00001900616D1F73197CF01089588279927DF
:1048C0000895FB01DC0104C08D910190801921F451
:1048D00041505040C8F7881B990B0895F894FFCFBA
:1048E0002E158415651561155D152D150102010143
:1048F00001131415161718191A1B1C818283E20064
:10490000E900EA00B500B600B700CD008301CC0095
:104910008A01920194012102230224022502260227
:1049200027022A02B300B4006F00700066363534E7
:104930009796949593929190F0F1F4F5F6F767308D
:1049400031000102020202060606090909090909E5
:104950000F0F0F12131313131313131313131D1E1F
:00000001FF
